:020000040000FA
:060000000FEF0BF01200EF
:060800000FEF0BF01200E7
:06082A0001004B16000066
:08083000FD00000003000000C0
:08083800040120511F0B01080F
:1008400001E05BD02051600BE842E842E842E84218
:10085000E842010801E051D0245103E0240501E001
:100860004CD02151230A48E0010A40E0030A30E05D
:10087000010A25E0240A22E0070A1FE0010A1CE021
:10088000030A11E0010A01E038D00101030E0B6FE9
:100890000101F50E0C6F000E0D6F010113930101A4
:1008A000080E106F2AD00101030E0B6F0101F50E27
:1008B0000E6F000E0F6F21D020D01FD01ED001016F
:1008C000030E0B6F0101EA0E0E6F000E0F6F15D0B5
:1008D0000101030E0B6F0101EA0E0C6F000E0D6F8C
:1008E000010113930101070E106F07D00101030EE0
:1008F0000B6F22C4F1F001D000D012000001EA6BAE
:10090000C20EEB6F010EEC6FED6BEE6BEF6B080E32
:10091000F06FE36BE26B1A0E726E1E0E736E0401C3
:10092000000E166F050E176F400E146F0401196F3D
:10093000080E1A6F050E1B6F880E186F0401480E03
:100940001E6F050E1F6F400E1C6F1200D9CFE6FF01
:10095000E1CFD9FF0001E26B040118BF30D0FC0EDB
:10096000DBCF02F01951D880025403E2FC0E19C407
:10097000DBFF0001E26BFC0EDB50E25D19E2E251AD
:10098000EA6A080FE96E050EEA22EF50E66EE251C0
:10099000E76EFD0EDBCFE9FFFE0EDBCFEAFFE7508F
:1009A000E926000EEA22E552E750EF6EE22BE3D78C
:1009B0000401400E196F1817187D880E18130001D6
:1009C000E25100D0E552E7CFD9FF1200D9CFE6FFC0
:1009D000E1CFD9FFE6520001E35101E02FD0DF6AF9
:1009E000DF2ADF50026E036AFF0E021801E1035096
:1009F00001E10BD0FD0EDBCFE9FFDB2AFE0EDBCFE2
:100A0000EAFF01E3DB2AEF50EBE1DF50026E036AFD
:100A1000D950FD0FE96EFF0EDA20EA6E0250EE5E4D
:100A20000350ED5AFD0EDBCFE4F0FE0EDBCFE5F018
:100A3000DFCFE8F00001E96B010EE36FE552E5520C
:100A4000E7CFD9FF1200D9CFE6FFE1CFD9FFE652B9
:100A50000001E35101E030D0DF6ADF2ADF50026E8F
:100A6000036AFF0E021801E1035001E10CD0FD0EF4
:100A7000DBCFF6FFDB2AFE0EDBCFF7FF01E3DB2A3D
:100A80000800F550EAE1DF50026E036AD950FD0F0D
:100A9000E96EFF0EDA20EA6E0250EE5E0350ED5A68
:100AA000FD0EDBCFE4F0FE0EDBCFE5F0DFCFE8F0AC
:100AB0000001010EE96FE36FE552E552E7CFD9FF80
:100AC0001200D9CFE6FFE1CFD9FFE65204011CBFE7
:100AD0006BD0030E0001E35D01E1E36BE35101E143
:100AE00063D0020EE35D06E104011D6B0001030EFD
:100AF000E36F54D0E30552E1400E026E036AE85101
:100B0000025C000E035803E2400EDF6E02D0E8C024
:100B1000DFFFDFCF1DF4DF50E85DE86F480EE66FC2
:100B2000050EE76FE90515E1DF5012E0E4C0F6FFBE
:100B3000E5C0F7FF0800F550E6C0E9FFE7C0EAFFAF
:100B4000EF6EE62B000EE723E42BE523DF06ECD760
:100B500013D0DF5011E0E4C0E9FFE5C0EAFFEF5039
:100B6000E6C0E9FFE7C0EAFFEF6EE62B000EE723E1
:100B7000E42BE523DF06EDD7E85110E104011D5118
:100B8000026E036A400E021801E1035004E1000105
:100B9000020EE36F03D00001030EE36F400E040169
:100BA0001C171C7D880E1C13E552E552E7CFD9FFB8
:020BB000120031
:0E0BB20004012051600BE842E842E842E842AC
:100BC000E842000901E055D02151070A51E00B0A23
:100BD0004FE0070A40E0010A2CE00B0A28E0020A75
:100BE00026E0030A22E0080A12E0010A0EE00F0ADA
:100BF0000AE0030A01E03CD00101010E0B6F010184
:100C0000040E126F36D036D834D090D832D00101CD
:100C1000010E0B6F0101140E0C6F010E0D6F01011F
:100C200013930101010E106F24D0A8D822D0F4D85C
:100C300020D00101010E0B6F0401245101010C6F42
:100C40000D6B150E0C27010E0D23010113930101ED
:100C5000010E106F0ED00101010E0B6F0401245123
:100C6000EA6A150FE96E010EEA2222C4EFFF01D0F5
:100C700000D01200800E0401205D57E12351030AC9
:100C800034E0010A10E0030A01E04DD00101010E39
:100C90000B6F01018A0E0C6F140E0D6F120E010105
:100CA000106F116B40D00101010E0B6F0401225136
:100CB000F66EF76AD890F636F7363F0EF626150E22
:100CC000F7220900F5CF0CF10A00F5CF0DF1020E65
:100CD0000101F76A0C25F66E0D51F7220900F5CFD8
:100CE00010F10A00F5CF11F11ED00101010E0B6FBA
:100CF00004012251F66EF76AD890F636F736430EA5
:100D0000F626150EF7220900F5CF0CF10A00F5CFF3
:100D10000DF10CC1F6FF0DC1F7FF0800F550010100
:100D2000106F116B00D00101138312000101010E3D
:100D30000B6F0F0EE66E710EE66E0F0EE66E87EC11
:100D400009F0E552E552E552010EE66E150EE66E2B
:100D5000010EE66E87EC09F0E552E552E55222C439
:100D600014F10401225104E10101050E126F05D0B6
:100D70000101060E126F7EEC04F012000401286BD4
:100D8000296B040120511F0B020A14E0030A0EE034
:100D9000010A01E033D00101010E0B6F040128812B
:100DA000010113A102D00401288328D00101010E02
:100DB0000B6F24D00101010E0B6F040124510F0BA6
:100DC000080DF350036A000F026E040E0322245133
:100DD000800B01E0010E040DF350010102240E6F9F
:100DE000000E03200F6F0EC1E9FF0FC1EAFFEF50A5
:100DF000040B03E00401010E286F00D001010B0574
:100E00000AE10101280E0C6F040E0D6F010113930E
:100E10000101020E106F12000401220510E12051A1
:100E20001F0B00090CE10101010E0B6F030E040101
:100E3000215D03E10101138102D00101139104013D
:100E400022513AE120511F0B020836E124510F0BC9
:100E5000000932E00101010E0B6F040124510F0B58
:100E6000080DF350036A000F026E040E0322245192
:100E7000800B01E0010E040DF350010102240E6FFE
:100E8000000E03200F6F030E0401215D07E1840EA5
:100E90000EC1E9FF0FC1EAFFEF6E0ED024AF06D0FE
:100EA0000EC1E9FF0FC1EAFFEF6A06D0880E0EC13E
:0A0EB000E9FF0FC1EAFFEF6E120028
:060EBA006C5002E0000E86
:100EC00001D0010E00090BE0040100513C0BE84287
:100ED000E8420D0802E10CD801D040D808D06C508F
:100EE00002E0000E01D0010E040901E047D8120013
:100EF000D9CFE6FFE1CFD9FFE65201010A6B0B6BB8
:100F0000106B116BD9EC05F0DF6ADF50026E036ADB
:100F1000010E025C000E03581BE201010B5101E0BF
:100F200017D0F76ADF34FE0BF736F66E490EF62659
:100F3000150EF7220900F5CF02F00800F5CF03F0F7
:100F400004D003C0FAFF0250F96EFBDFDF2ADDD7C1
:100F5000E1D8E552E552E7CFD9FF1200020E0101B8
:100F60000A5D0AE198D8040100BD03D0C80E006FE5
:100F700002D0880E006F01D013D91200040E0101B7
:100F8000125D0AE122C46EFF6E50000803E2050EF6
:100F9000126F02D0030E126F01010A050AE10BD88D
:100FA000040104BD03D0C80E046F02D0880E046F84
:100FB00001D0F6D81200D9CFE6FFE1CFD9FF020E5B
:100FC000E1260101080E105D000E115905E210C165
:100FD000DEFF11C1DDFF03D0080EDE6EDD6A040105
:100FE00004930491010EDB500413DFCF05F4000ECF
:100FF000DB500101105F010EDB50115B280E0E6FFC
:10100000040E0F6F010113A31ED0D9CFE9FFDACF71
:10101000EAFFEE50ED1016E00CC1F6FF0DC1F7FF30
:101020000800F5500EC1E9FF0FC1EAFFEF6E0101A4
:101030000E2B000E0F230C2B0D23DF06010E01E2F9
:10104000DB06E3D71CD0D9CFE9FFDACFEAFFEE50B9
:10105000ED1015E00CC1E9FF0DC1EAFFEF500EC124
:10106000E9FF0FC1EAFFEF6E01010E2B000E0F2307
:101070000C2B0D23DF06010E01E2DB06E4D7F56E33
:10108000020EE15C02E2E16AE552E16EF550E552E2
:10109000E7CFD9FF1200D9CFE6FFE1CFD9FF020E8B
:1010A000E126030E04010015E76E010EE7CFDBFF1A
:1010B00001C4DFFFDE5001011027DD501123280E8F
:1010C0000C6F040E0D6FD9CFE9FFDACFEAFFEE50B7
:1010D000ED1014E00CC1E9FF0DC1EAFFEF500EC1A5
:1010E000E9FF0FC1EAFFEF6E0E2B000E0F230C2B52
:1010F0000D23DF06010E01E2DB06E5D7F56E020ED9
:10110000E15C02E2E16AE552E16EF550E552E7CFBB
:10111000D9FF120001010B510CE10401080E016F0F
:10112000200E026F040E036F840E006F0401046F23
:1011300035D0040120AF22D0010110510401265DF9
:10114000010111510401275904E226C410F127C4FA
:1011500011F131DF0101010E0A6F0401080E016F68
:10116000200E026F040E036F800E006F0401280E24
:10117000066F040E076FC80E046F10D00101020E37
:101180000A6F0401056BC80E046F0401080E016F9D
:10119000280E026F040E036FC80E006F6D981200C8
:1011A00001010A6B0401080E016F200E026F040E8C
:0C11B000036F880E006F0401046B120036
:0411BC006DA60FD835
:1011C00002D06DB613D80101120508E16DBA06D040
:1011D000686A696A69806988020E126F12006D6A16
:1011E000696A6D860101010E126F12006D6A696AEB
:1011F0000101126B1200F6EF08F00101125101E13A
:101200003AD06850040B04E06950040B01E03CD86C
:101210006DB231D06850010B04E06950010B01E060
:1012200054D86850100B04E06950100B01E024D82A
:101230006850400B04E06950400B01E03BD8685017
:10124000200B04E06950200B01E036D86850020BF7
:1012500004E06950020B01E036D8030E0101125D73
:1012600001E209D06850080B06E06950080B03E062
:101270005DEC07F068961200698468986D82A19A07
:10128000A08A0300A09A12006D92699468941200DB
:10129000010113A10ED0F8DF6D840101080E166F55
:1012A000070E176F1607000E175B16511711FAE19C
:1012B0006D941200689C120070A003D0D0EC08F06E
:1012C0007090689A1200689212006A6A686A9F0EAB
:1012D0006B6E7B0E696E6E6A0F0EE66E710EE66EB9
:1012E0000F0EE66E14D8E552E552E552160E706EFA
:1012F00068A602D06896FCD76D98D0EC08F0010182
:1013000013910101146B0101030E126F1200D9CF6A
:10131000E6FFE1CFD9FFFD0EDBCFE9FFFE0EDBCF0D
:10132000EAFFFC0EDB5004E0EE6AFC0EDB06F9D7A8
:08133000E552E7CFD9FF1200DE
:08133800FC0E8B169416948440
:101340008250040B01E0010E0001606F896A92680F
:101350008A68936A1200D9CFE6FFE1CFD9FFE6523F
:10136000DF6A4DD8060E0101125D03E36D50020BDA
:1013700001E040D0200EE66E610EE66E000EE66ED5
:10138000A6EC04F0E552E552E552DF6EDFCF02F045
:10139000000EE76E0218E8AE02D0023403D0E75028
:1013A000D880025427E261C08AFF8B720001FD5190
:1013B0000EE00001E3510AE10001FD6B360EE66E1E
:1013C000160EE66E23EC05F0E552E55213D000014F
:1013D000E35110E180CFA1F00001A26B0001A10E4A
:1013E000E46F000EE56F0001010EE86F0001E96B8C
:1013F0000001E36FE552E552E7CFD9FF120000018B
:10140000FE51FF1104E1500EFE6FC30EFF6FFE0789
:10141000000EFF5B6DA205D0FE51FF1101E18B9024
:1014200020D00101125102E18B901BD0120502E184
:101430008B8017D0020E125D02E18B8012D0030E5A
:10144000125D02E18B800DD0050E125D02E18B80F2
:1014500008D0060E125D05E10001FE51FF1101E109
:101460008B7012008250040B01E0010E0001605DE0
:1014700009E08250040B01E0010E606F82B402D0DB
:0A148000010E02D0000E00D0120091
:06148A0012010002020045
:101490000008D8040A00000001020001090243000C
:1014A00002010080FA090400000102020100052483
:1014B0000010010424020205240600010524010095
:1014C000010705820308000209040100020A000066
:1014D00000070503024000000705830240000004E6
:1014E00003090434034D006900630072006F006358
:1014F0000068006900700020005400650063006807
:10150000006E006F006C006F0067007900200049DA
:10151000006E0063002E0028035500420057002093
:10152000004600690072006D00770061007200657E
:1015300000200043002000760030002E0031009C87
:0B154000149C14DF14E3141715380886
:04154C002A0EF66EFF
:10155000080EF76E000EF86E01010900F550056FD8
:101560000900F550066F03E1056701D03DD0090081
:10157000F550006F0900F550016F0900F550026F3A
:1015800009000900F550E96E0900F550EA6E0900FE
:1015900009000900F550036F0900F550046F0900B8
:1015A0000900F6CF07F1F7CF08F1F8CF09F100C134
:1015B000F6FF01C1F7FF02C1F8FF0101035302E189
:1015C000045307E00900F550EE6E0307F8E2040744
:1015D000F9D707C1F6FF08C1F7FF09C1F8FF0101FC
:0A15E0000507000E065BBFD71200DE
:0615EA0005D810D8ABEC9F
:1015F00009F0FCD712000F0EC112140E6F6E01011C
:10160000126B0101136B0101146B9CEF09F0DEEC0E
:0E16100008F06FBE02D0FDEC08F061EF05F0AF
:02161E0013EEC9
:1016200000F023EE00F0F86A019CA6EC0AF0F5EC5D
:061630000AF0FDD71200D4
:0A163600554257204669726D776136
:0B164000726520432076312E300D0033
:03164B000100009B
:00000001FF
